:0400000080314928DA
:1000060001347E1480312100911E0A280B284728CE
:100016002000911E0F281028472823001908F000F9
:1000260070082000C0000D30400603191B281C284C
:10003600252800302502403003192402031C2428F9
:10004600252837280130F0007008BB002408A03EA0
:100056008600870181012508A7002408A600A401BF
:10006600A5012100911247284008F0002408A03E6F
:1000760086008701700881000130A4070030A53D85
:100086002508A7002408A6007E10090080314B2809
:10009600803103208031EF00FC01203084000030E5
:1000A600850041308F31F1278031A0308400003047
:1000B600850040308F31F1278031203084000130B7
:1000C600850050308F31F12780317E10200080313D
:1000D6006C28F230210099009801163097000630FE
:1000E6002000EE001330ED00AD30890B7828ED0BC3
:1000F6007828EE0B7828003287313E278031873109
:10010600C62780313F302000B0000030B100B40176
:10011600B5013408A03E8600870181010130B4078D
:100126000030B53D003035023F3003193402031C60
:100136009D289E288C28B401B5013408413E8600CE
:10014600870181010130B4070030B53D003035022A
:100156001F3003193402031CB128B228A028B401A9
:10016600B5013408203E8600013087008101013048
:10017600B4070030B53D003035024F300319340264
:10018600031CC628C728B4282030ED006D08BA0025
:100196008F31F72780318F31F72780318630F10094
:1001A6008530F2008631C62680311030F100873066
:1001B600F2008631C6268031D330F1008730F20056
:1001C6008631C6268031DF30F6008730F70085316C
:1001D6005825803120308731EB278031F530F60005
:1001E6008730F7008531582580316630F100873039
:1001F600F2008631C626803138302000E900093009
:10020600EA000A30EB000030EC0041308631072668
:1002160080314130F6000030F700853158258031B5
:100226008F31F7278031BE30F1008430F2008631FD
:10023600C62680315230F1008430F2008631C6265F
:1002460080314C30F1008630F2008631C62680318E
:100256008F31F72780318C30F1008630F2008631FD
:10026600C626803130302000ED006D08FC002200EB
:100276000C1606302000EE001330ED00AD30890B71
:100286004229ED0B4229EE0B422900327C088731C8
:10029600EB27803122000C1206302000EE001330CE
:1002A600ED00AD30890B5529ED0B5529EE0B55297F
:1002B600003201302000ED006D08FC0739307C0269
:1002C600031C662967293A298F31F72780318B135A
:1002D600230019082000ED006D08C00023001D163C
:1002E6000B088B130B17B930F1008730F2008631FB
:1002F600C6268031653020009B009A019110183087
:100306009C005330F1008730F2008631C6268031DA
:10031600250093013F3093051308F0390C389300FC
:1003260020001C1521000C118F31F72780318A30EF
:10033600F1008730F2008631C62680312030F10088
:100346000030F2008731272780312030F1004E300F
:10035600F2008631AA2680312730F1008530F2007E
:100366008631C62680318830F1008430F20086312D
:10037600C62680312000B401B5011030B20000302D
:10038600B300492A8531DE2580318B1706302000DF
:10039600EE001330ED00AD30890BCF29ED0BCF29E0
:1003A600EE0BCF29003220003B03031DDB29DC299D
:1003B600372AFE30F1008730F2008631C6268031BA
:1003C600A030F6000030F7008531582580318F3196
:1003D600F72780310B30F1008830F200A030200082
:1003E600ED006D08F3008531B32580317108720484
:1003F6000319FE29FF29372AA4308331302380319F
:1004060078082000B3007708B200320833040319D5
:100416000D2A0E2A372A3308F2003208F1008731F6
:1004260027278031AA30F1008730F2008631C626B0
:10043600803120003308EA003208E9000A30EB0078
:100446000030EC0041308631072680314130F6001D
:100456000030F7008531582580310530F1008830AD
:10046600F2008631C62680318B13031020000C1E45
:10047600031403183F2A422A22000C16442A22009B
:100486000C1201302000B4070030B53D01303302B4
:100496000030031932020318512A522A5B2A00300F
:1004A6003502783003193402031C5A2A5B2AC529FF
:1004B600230019082000ED006D08C0008B13C00151
:1004C6002A30F1008630F2008631C62680319A3015
:1004D600F1008730F2008631C62680311030F100F7
:1004E6000030F2008731272780312030F1004E306E
:1004F600F2008631AA2680312000B201B301F9301C
:10050600F1008630F2008631C62680310030F100D7
:10051600F20087312727803130302000ED006D084A
:10052600FC00B001B101EF01EF0A6E30ED003208B8
:100536006D02B00033090318890AB1003108F200D0
:100546003008F1008631AA2680317C088731EB27F6
:10055600803101302000ED006D08FC073A307C0246
:10056600031CB62AB72A1D2B09308731EB278031A9
:1005760030302000ED006D08FC003308EA00320838
:10058600E9000A30EB000030EC00413086310726E6
:1005960080314130F6000030F70085315825803132
:1005A60009308731EB27803120003108EA00300816
:1005B600E9000A30EB000030EC00413086310726B6
:1005C60080314130F6000030F70085315825803102
:1005D6008F31F72780312000320825009100200056
:1005E6006F08ED00EE01ED1BEE0332086D07B20059
:1005F60033086E3DB30032083304031D032B042B6E
:10060600112BEF01EF0A03100C1E031403180C2B19
:100616000F2B22000C16112B22000C12003020008A
:100626003302643003193202031C1A2B1B2B1D2BB9
:10063600EF01EF03911E202B212B272B23001908F6
:100646002000ED006D08C00052304006031D2C2B23
:100656002D2B982A0100803149282000E800372BED
:100666000130E1006108E80768088600870120304C
:10067600010603193F2B402B332B680886008701A0
:10068600093001060319482B492B332BE601E701F4
:10069600E5016808860087012D300106031D542BED
:1006A600552B5E2B0130E1006108E5070130E100C2
:1006B6006108E8078C2B6808860087012B30010645
:1006C600031D662B672B8C2B0130E1006108E807C0
:1006D6008C2B20006808860087010108E100E201F2
:1006E6006708F2006608F1000A30F3000030F400F3
:1006F60086316D268331200061087107E3006208A8
:10070600723DE4006308D03EE600FF30643DE7003A
:10071600672B6808860087010108873178278331AF
:100726000318962B972B6C2B2000650803199C2B1E
:100736009D2BA92B6609E1006709E200E10A03196E
:10074600E20A6108F7006208F800AD2B6708F800B6
:100756006608F70008002000E8006208E600610865
:10076600E5006408F2006308F1006608F400650815
:10077600F30084311624833172082000E6007108E4
:10078600E5000130F9007908E80765086604031DED
:10079600CD2BCE2BB42B6808860087018101013052
:1007A600E8026408F2006308F1006208F4006108D8
:1007B600F3008431F32483317108F90079082000AD
:1007C600E7006408F2006308F1006208F4006108BB
:1007D600F30084311624833172082000E200710888
:1007E600E1000A306702031CF92BFA2BFE2B0730B7
:1007F600F9007908E7073030F9007908E707670854
:10080600F900680886008701790881000130E8024E
:1008160061086204031D102C112CD42B0130F90041
:100826007908E8070800F701F8017108720403194E
:100836001D2C1E2C4D2CF601F60A2A2C0130F13502
:10084600F20D890B222C0130F5007508F607F21F10
:100856002D2C2E2C212C0130F735F80D890B2F2C41
:1008660072087402031D392C71087302031C3C2C98
:100876003D2C422C7108F3027208F43B77140130C8
:10088600F236F10C890B432C0130F602031D4C2C79
:100896004D2C2E2C7808F2007708F1000800203441
:1008A600553441345234543431342034483461346C
:1008B60072346434773461347234653420342034CD
:1008C60031343934323430343034203452344134D3
:1008D60031342034503469346E3436343D34523435
:1008E600583420342C3420342034523441343034BB
:1008F6002034703469346E34203437343D34543403
:10090600583420340D340A340034203473346934B6
:100916002034503457344D343E3432343534353443
:1009260020346F34753420343E343134323430342C
:10093600203462346F34753463346C346534733404
:1009460028343634303473346534633429343D34D2
:100956003E34203420346D346F34643465342034AE
:100966006734693472346C3461346E34643465349B
:100976000D340A340034203448346134723464341B
:10098600773461347234653420343A34503449341F
:1009960043343134323446343134383434343034F8
:1009A60020344434693470343834203420344634A6
:1009B6004F3453344334203469346E3474346534DC
:1009C60072346E34653420343D3438344D34483412
:1009D6007A3420347834343420340D340A340034F4
:1009E600710872040319F82CF92C222DF601F60A67
:1009F600052D0130F135F20D890BFD2C0130F50086
:100A06007508F607F21F082D092DFC2C72087402D2
:100A1600031D0F2D71087302031C122D132D172DA4
:100A26007108F3027208F43B0130F236F10C890BBF
:100A3600182D0130F602031D212D222D092D7408D3
:100A4600F2007308F10008002034433468346F3430
:100A56006934783420346D346F346434653420342A
:100A6600503457344D34203476346934613420346C
:100A76005434653472346D3469346E3461346C3494
:100A860020344B346534793462346F3461347234D3
:100A9600643420342034503457344D343D34783463
:100AA600783478340D340A3400347708F200760846
:100AB600F1008631E026853172082000A100710818
:100AC600A000A201A301772D76082000220784004A
:100AD6007708233D850000088731EB2785310130F3
:100AE6002000A2070030A33D2308803AF800210821
:100AF600803A7802031D812D20082202031C842DD2
:100B0600852D672D08002034503472346F346A34D2
:100B16006534743420344D3450344C3441344234CA
:100B2600583420343A3447347534693472346C346A
:100B360061346E34643465345F34503457344D3424
:100B46005F3431343234463431343834343430342A
:100B56005F3432343034323432340D340A340034B3
:100B6600BC2D0130F1070030F23D0130F40074086D
:100B7600F3077308860087017108840072088500F0
:100B86000008F40001087402F5007508F6007608FE
:100B9600031DCE2DCF2DD82D710884007208850037
:100BA6001200031DD72DD82DB42D7608F100F201C1
:100BB600F11BF203080023001908F1007108200058
:100BC600C000A401A501003025023F30031924020C
:100BD600031CEE2DEF2DF02DFA2D2408A03E8600E5
:100BE600870181010130A4070030A53DE62DC00133
:100BF6002100A0012000BB01A401A501A601A701B7
:100C0600C001210091160800FB002000EA1F0C2EEF
:100C16000D2E1D2E2D30FA007B08860087017A08DE
:100C260081000130FA007A08FB07E909EA09E90AB6
:100C36000319EA0A6A08E2006908E1006C08E400A0
:100C46006B08E3007B088331AE238631080020342D
:100C5600433468346F346934783420346D346F34F7
:100C660064346534203447347534693472346C34F2
:100C760061346E34643465340D340A3420345234AD
:100C86003D34523465347334653474340D340A3467
:100C960000342034503457344D34203473346F3498
:100CA6007234743469346534203450343134413408
:100CB60020347334753472342034703469346E34AD
:100CC60020343534203452344134323420340D3417
:100CD6000A340034F501F601711C722E732E772E3C
:100CE6007308F5077408F63D0130F335F40D890BEA
:100CF600782E0130F236F10C890B7D2E71087204C4
:100D0600031D862E872E6F2E7608F2007508F100D9
:100D1600080020344334683465346B3420344C3452
:100D26006534643420346F346E34203452344134A4
:100D36003434203461346E346434203455344134D0
:100D460052345434323420340D340A340034F4012D
:100D5600F501F401F501B72E4230890BB02E0032B1
:100D66000130F4070030F53D7508803AF30072084B
:100D7600803A7302031DC12E71087402031CC42E2F
:100D8600C52EAF2E0800D62E23009E1CCB2ECC2EB1
:100D9600C72E710884007208850000089A00013089
:100DA600F1070030F23D71088400720885001200D8
:100DB600031DDE2EDF2EC72E08007208F50071080F
:100DC600F400E92E0130F4070030F53D7408840084
:100DD600750885001200031DF12EF22EE52E71080E
:100DE6007402F1007208753BF20008002034733477
:100DF600653474342034643475347434793420346E
:100E06006434653420343034203461342034313451
:100E1600303430340D340A340034203456346534DA
:100E26007234733469346F346E3420343A34203477
:100E360032343034323432342D3431343234323484
:100E460035340D340A3400347208F4007108F300A6
:100E5600F436F30CF436F30C730825009100710890
:100E66000339F3000430F335890B362F1308CF39D5
:100E760073049300080022009D018C01EB302100D1
:100E86008C0023008C0124008C0121000C150C120F
:100E960022000C1224000C160C15210095170800D0
:100EA600203449346E346934743420344E346F340B
:100EB60072346D3461346C342034503457344D34CC
:100EC6000D340A3400342C3420342034583443345E
:100ED60038342034763465347234733469346F347C
:100EE6006E3420343A3420340034F200F1013A30C2
:100EF600720203187F2F802F882F30307202031C56
:100F0600852F862F882FF101F10A710C08002034F5
:100F160073346534743420346434753474347934F9
:100F260020343D34333432340D340A340034203422
:100F360073346534743420346434753474347934D9
:100F460020343D34313436340D340A3400344E34D2
:100F5600653477342034503457344D342034763465
:100F660061346C34753465342034003420344934AB
:100F76006E3469347434203454344D34523432343B
:100F86000D340A34003421009112083023009F00EA
:100F960090309D0024309E0067309B009C01080025
:100FA600203443346F346D34703469346C346534B2
:100FB60020343A34203400344434653463342034E5
:100FC600323435342034323430343234323400342E
:100FD600F1002000111EF02FF12FEC2F71082300D5
:100FE6009A000800313438343A34313437343A34DC
:100FF6003434323400345234653463347534203436
:101006003A34003420344F346B340D340A3400340F
:0A101600503457344D343D3400349B
:101FE200640080010131890BF22F00340D308731FA
:0E1FF200EB278F310A308731EB278F31080043
:020000040001F9
:08000000FF3FFF3FFF3FFF3F00
:04000E00E43FFF3F8D
:00000001FF
